:100000000C942A000C9447000C9447000C94470071
:100010000C9447000C9447000C9447000C94470044
:100020000C9447000C9447000C9447000C94470034
:100030000C9447000C9447000C9447000C94470024
:100040000C9447000C9447000C9447000C94470014
:100050000C94470011241FBECFE5D4E0DEBFCDBF16
:1000600010E0A0E6B0E0E0E6F1E002C005900D92FD
:10007000A036B107D9F710E0A0E6B0E001C01D92AC
:10008000A036B107E1F70E9477000C94AF000C9402
:10009000000081E088BB87BB12BA81BB08959B0139
:1000A000AC0194E0220F331F441F551F9A95D1F7DE
:1000B00060E876E988E990E00E948D0021503040A8
:1000C000832F992780BD29B98AB188618AB980B503
:1000D000866880BD08955F9903C080E090E0089530
:1000E0008CB1992708955D9BFECF8CB9089581E06E
:1000F00088BB87BB12BA81BB60E875E280E090E004
:100100000E944F005F9BFECF8CB19927282F882338
:10011000C9F35D9BFECF2CB9F5CFA1E21A2EAA1B25
:10012000BB1BFD010DC0AA1FBB1FEE1FFF1FA217A7
:10013000B307E407F50720F0A21BB30BE40BF50BA4
:10014000661F771F881F991F1A9469F7609570952D
:10015000809590959B01AC01BD01CF010895FFCF23
:00000001FF
